:020000040800F2
:1010000038390020D1100008754300086923000812
:1010100000000000000000000000000000000000D0
:10102000000000000000000000000000E14F000888
:101030000000000000000000454400081D550008A5
:10104000E310000800000000E3100008E3100008AF
:10105000E3100008E3100008E3100008E3100008A4
:1010600000000000E3100008C51500086516000820
:10107000E3100008E3100008E3100008000000007F
:10108000E310000825560008E3100008E3100008EC
:10109000E3100008E3100008E3100008E310000864
:1010A000E3100008C54F0008E31000083D56000893
:1010B000C5560008115700080348854600F03AF964
:1010C00000480047F9650008383900200844F04717
:1010D0000448804704480047FEE7FEE7FEE7FEE7D6
:1010E000FEE7FEE7C9550008B910000830B50B4609
:1010F000014600202022012409E00D46D5409D42F2
:1011000005D31D469540491B254695404019154677
:10111000521E002DF1DC30BD70B50024254600289C
:1011200001DA01244042002901DA01254942FFF792
:10113000DDFFAC4200D04042002C00D0494270BDDF
:10114000F8B500242546002904DA0E4601240021C2
:101150004042B141002B04DA1E46002352420125D1
:10116000B34100F076F88C4617461E46AC4203D0D9
:10117000002540428D41AC46002C02D0002657424B
:101180009E4161463A46334601B0F0BD10B5202A73
:1011900004DB0846203AD040002110BD0B46D34066
:1011A000D0402024A21A91400843194610BD03469E
:1011B0000B439B0703D009E008C9121F08C0042A8B
:1011C000FAD203E00B780370401C491C521EF9D27E
:1011D0007047D2B201E00270401C491EFBD270473A
:1011E0000022F6E710B513460A4604461946FFF7F3
:1011F000F0FF204610BD0321001D401E037812029F
:101200001A43491EF9D510467047C217C10F504006
:1012100010B54018CA079623002100F052F810BDFF
:10122000C20F410040020123400ADB05D207090E2C
:10123000C0187F2901DA00207047962903DC962325
:10124000591AC84001E096398840002AF4D040423B
:101250007047F0B51FB40646002082B00546402412
:10126000019100901BE0019922460F463046FFF79E
:101270008DFF049A059B801A994110D31046194698
:10128000224600F069F8361A8F4101972246012064
:101290000021009F00F060F838184D410090204672
:1012A000641E0028DFDC019B00982946324607B007
:1012B000F0BD002904DA401C490001D1400840007B
:1012C000704770B40024050C05D11024000402D12D
:1012D000002921D01124050E01D100020834050F88
:1012E00001D10001241D850F01D18000A41C00281C
:1012F00001DB4000641C002908D020252E1B0D4670
:10130000F540A14000D001212943084301061B1BE1
:10131000000ADB1D02D5002070BC7047DB051818E1
:1013200080180029F8DA401C4900F5D170BC40084B
:1013300040007047064C0125064E05E0E36807CCE7
:101340002B430C3C98471034B442F7D3FFF7B8FE58
:101350001C7200083C72000810B5202A04DB01460C
:10136000203A9140002010BD914020239C1A034652
:10137000E3401943904010BD70B58D180478401CAF
:10138000A207920F01D10278401C231106D10378E5
:10139000401C03E006780E70401C491C521EF9D117
:1013A000002B15D002780C268A1A3440401C0C2CD5
:1013B00003D0A401121B9B1C08E004782402121B1A
:1013C000401CF8E714780C70491C521C5B1EF9D5C0
:1013D000A942D3D3002070BDF0B51C4CA0684007D3
:1013E000C00F31D1206C1B4D82B219481A490369D4
:1013F0000120DE07002E0AD08A82184B18492846A1
:101400009A4201D2012200E000220A6012E09D43CC
:1014100006D0144D9D4306D0134D9D4306D009E0E0
:101420000A83124806E00A84114803E04A84114AFC
:10143000528BCA834103490BA162A1680E4A114035
:10144000091DA160024908610020F0BD002401408F
:10145000C000002000010020C419002098080000EE
:10146000640100200000014000000244000001C0AF
:10147000000002C4A0F7FF1FE8FFFF7FF0B51E4F7A
:1014800085B03D691D4C6D1C3D612668A4680294C1
:1014900000966C4665800190218162810393386AD1
:1014A00001011748091800220B4610461C5CFF2C4E
:1014B00004D1401C1028F9D3002A17D01022684606
:1014C00000F00CF9386AF861401C38620001012113
:1014D00009031030884201D900203862F8680949B0
:1014E000401CF8604867002005B0F0BD1022684637
:1014F00004F0A8FBE6E7000040010020E46D0008CE
:1015000000D0000844190020002911D08268521828
:1015100082604368934200DCD21A00238361C3686F
:10152000934201D101234361826002695218026132
:1015300008467047F0B50020174D0127144B154C95
:101540003F03E86017E0625A144EB24212D1EA68D3
:101550000919521CEA604A882E69B24205D92A61EB
:10156000E8614A686A61421C2A624988994201D24C
:101570000B46A861401C0101B942E4D3286A00016E
:101580001030B84201D900202862E868F0BD0000A0
:10159000FFC99A3B00D0000840010020AA55000076
:1015A00010B50421054800F0BCF805480021816110
:1015B000C1610161C1600162084610BD00D0000830
:1015C0004001002070B5234DE86A401CE862224CBF
:1015D00020688006C00F11D02868296B4018286049
:1015E000296B28465830064600F058F820206060E5
:1015F000B06900280AD0002028636872206880053E
:10160000C00F02D001204002606070BD304600F083
:1016100075F912494A78A3585B085B00A350F36838
:1016200032684E78D2180C4B0C33F2500A4B4A7881
:101630001B1DD658360C36040643D65049786258DE
:1016400001231A43625028630548816880221143B0
:101650008160D3E7E408002000000240FF71000829
:10166000003801400B49C86A401CC8620A48026839
:101670009204D20F05D001225203426000220A6375
:101680004A7201688903C90F02D0012149044160EF
:1016900070470000780900200000024010B50029C2
:1016A00010D0C26843685218934200DCD21A00235B
:1016B0004361C2608468944204D1012282618360E4
:1016C000C360C361084610BDFF2109220131D20663
:1016D000002801D09162704791617047F0B585B0E4
:1016E00016460D46074600F06FFA701E800A401C31
:1016F000029000200090019503A9684600F0CCF903
:101700000024760807E060003A5A411900230120BE
:1017100000F01CFA641CA642F5D800F00DFA05B0E2
:10172000F0BD7FB50D46044600F04EFA00206A4633
:1017300031C203A9684600F0AFF900F0FDF904B02A
:1017400070BD000006490020C861064801690422F6
:10175000114301610169402211430161704700009A
:101760001835002000200240064A0021D1610649B8
:101770000A6902231A430A6148610869402210433A
:1017800008617047183500200020024010B5054B55
:101790000022DA61044A13690124234313610180A2
:1017A00010BD0000183500200020024010B50B4A83
:1017B0000020D168CB060A4904D5C8690223184322
:1017C000C8611020D3685B0705D5CB69012423438A
:1017D000CB6104210843D06010BD0000002002400E
:1017E0001835002070B5044600F000FA0546104E8A
:1017F0000AE0601C08D0002C04D000F0F7F9401B70
:10180000A04201D9032070BDF068C007F1D1F06893
:10181000800601D52020F060F068C00602D4F06890
:10182000400703D5FFF7C2FF012070BD002070BD47
:10183000002002400A07120F01219140014201D00D
:1018400001207047002070470A07120F01219140C4
:10185000014201D00120704700207047F8B50B0508
:101860001B0E254C5B001C1909239B01E3180093F8
:101870000523DB01E618012307469B020A07E5184A
:101880000020120F3B0004F0CFFB09060A0E1219CC
:101890001D21282F2E00FF2928D800981BE0FF29A2
:1018A00024D8009808E0FF2920D8B08A18E08029C1
:1018B0001CD20F2080012018808E11E0802915D2C3
:1018C000A88A0DE0402911D2B08E09E040290DD23E
:1018D0000B2080010EE0808A02E0802906D2A88ECB
:1018E0001146FFF7B1FFF8BD802901D30020F8BDF4
:1018F0000920C0012018EEE7C4130020C1688268E7
:10190000914201DA501A7047914202DC4269002A82
:1019100002D04068401A704780690028FBD0002040
:101920007047C2688168914201DA501A704791424B
:1019300002DC8269002A02D04068401A7047406980
:101940000028FBD000207047064901228969120354
:1019500008180101914201D3FF3801380249000102
:10196000401870474001002000D0000800B5082052
:1019700000F07CFD00BD0000F0B5334C4B001C199D
:101980000923DB01E5180B230246DB010020E318E5
:10199000892A25D00EDC2C4F2C4B4E00F619F61858
:1019A000803A130004F040FB091F1F152125292E42
:1019B000333A15008D2A3FD00CDC8A2A33D08B2A8B
:1019C00035D08C2A05D140293ADA0B208001201825
:1019D000808EF0BD992A03D0A12A01D0FE2AF8D129
:1019E00080292DDA2EE00846F0BD102928DAB08AC9
:1019F000F0BD102924DAB08EF0BD102920DA0520C0
:101A0000C00108E008291BDA0F208001DFE7082960
:101A100016DA012080022018808AF0BD80290FDAB2
:101A20003420285EF0BD80290ADAA88AF0BD40295A
:101A300006DA0D208001CAE7402901DAA88EF0BD40
:101A40000020F0BD988EF0BDC413002040020000BD
:101A500010B5074A106A074B9969146AA04201D071
:101A6000106A9969044A51430914401A10BD0000D4
:101A70007001002000E000E05505000031B500F0E5
:101A8000B5F8009C0546601C00D0641C00F0AEF860
:101A9000401BA042FAD338BDF8B5054623480F468F
:101AA000017E012601290BD0012101762868204CF6
:101AB000012807D02046FFF795FE002813D030E01C
:101AC0000220F8BD2046FFF78DFE002829D1FFF740
:101AD00039FE2046FFF786FE0646164801690422B5
:101AE000914301611DE00020C04338606C6812E042
:101AF0002046FFF739FE0E48FFF774FE06460D48F4
:101B00000169022291430161002E01D03C6008E08E
:101B10000120C0022418A8686968C0024018A042C9
:101B2000E6D80248002101763046F8BD183500207D
:101B300050C3000000200240034801698022114385
:101B4000016100207047000000200240F0B51FB482
:101B500005461A480024017E16461F46012907D073
:101B6000012101761648FFF73DFE002803D021E051
:101B7000022005B0F0BD012D1AD0022D18D0042589
:101B800016E0220130463946FFF700FB81B201988A
:101B900062001018FFF7FAFD0948FFF723FE094914
:101BA0000A69520852000A61002803D1641CE4B299
:101BB000AC42E6D3014900220A76DAE71835002064
:101BC00050C300000020024005480169090605D500
:101BD000044941600449416000207047012070477A
:101BE0000020024023016745AB89EFCD0148006822
:101BF00070470000E007002002480168491C0160AE
:101C000070470000E007002010B506480168102268
:101C100011430160002000F007F800F017F80020E1
:101C200010BD00000020024010B5044600F040F94D
:101C30007D21C900FFF75AFA00F07AFB0022214605
:101C4000501E00F025F8002010BD000008B50F4818
:101C50008169012211438161816911400091C2694A
:101C600001040A43C261C069002208400090114685
:101C7000501F00F00DF800221146901E00F008F8E9
:101C800000221146501E00F003F808BD001002406B
:101C900010B502F09DFB10BDF8B504460068364D46
:101CA000C00354D5E8690026C00007D4E8692904B8
:101CB0000843E861E8690840012600902F48016860
:101CC000C90511D4014608688A1510430860FFF75A
:101CD0008DFF074604E0FFF789FFC01B642823D867
:101CE00026480068C005F6D5286A03210902084085
:101CF0001FD062680A4082421BD0286A2A6A884341
:101D0000012109040A432A622A6A8A432A62286254
:101D1000C0070ED0FFF76AFF074607E0FFF766FF30
:101D2000C11B1748814201D90320F8BD286A8007EA
:101D3000F4D5286A032109028843616808432862B0
:101D4000002E04D0E869012109078843E861207862
:101D5000C00705D0286BA16880088000084328636D
:101D60002078800605D5286B10218843E168084358
:101D700028630020F8BD0000001002400070004001
:101D800088130000F8B5044644480E460068C007B2
:101D9000C00FB0420AD241480168490849003143A6
:101DA00001600068C007C00FB0425CD120783C4F92
:101DB000800705D57868F0218843A16808437860DA
:101DC0002078C0073FD06068012813D03968022806
:101DD00013D08907002946DA796889088900014308
:101DE0007960FFF703FF0546606801280DD00228DF
:101DF00017D024E039688903ECE78901EAE7FFF7A7
:101E0000F5FE411B2748814217D878680007800FEC
:101E10000128F4D117E0FFF7E9FE411B2148814278
:101E20000BD878680007800F0228F4D10BE0FFF789
:101E3000DDFE411B1B48814201D90320F8BD7868B3
:101E40000007800FF3D115480168C907C90FB142D7
:101E50000BD9016849084900314301600068C00797
:101E6000C00FB04201D00120F8BD2078400706D550
:101E70007868072109028843E1680843786000F028
:101E80001DF87968084A0906090F515CC8400749DE
:101E900008600020FFF7C8FE0020F8BD00200240C7
:101EA000001002408813000004720008DC070020C4
:101EB0000148006870470000DC07002030B514A01E
:101EC0000FC889B06C460FC415A00FC80FC4184DB9
:101ED0006A680C2011460140164B042910D01648A0
:101EE00008290ED19102090F6C46645CE96A04ADC1
:101EF0000907090FD203695C920F022A03D003E09D
:101F0000184609B030BD1846FFF7F0F86043F8E70F
:101F100002030405060708090A0B0C0D0E0F10102A
:101F20000102030405060708090A0B0C0D0E0F1029
:101F300000100240001BB70000127A00FEB50446F4
:101F40000078D54DC00748D068680007800F012889
:101F500019D068680007800F022804D16868C003A0
:101F6000800F02280FD0012160680904012811D0D8
:101F70008A00002801D0052816D0286888432860E8
:101F80002868904308E02868800326D56068002808
:101F900073D022E02868084328606068002810D0C9
:101FA000FFF724FE064608E0286810432860F1E7A2
:101FB000FFF71CFE801B642870D828688003F7D5C3
:101FC0000BE0FFF713FE064604E0FFF70FFE801B51
:101FD0006428F1D828688003F7D420780126800788
:101FE00000283DDA68680007800F13D06868000792
:101FF000800F022804D16868C003800F012809D02F
:10200000E068002828681CD030432860FFF7EEFD08
:1020100007460BE0286880070BD5E06801282CD123
:1020200007E0FFF7E3FDC01B0228C5D8286880073A
:10203000F7D52868F82188432169C900084328603A
:102040000EE0400840002860FFF7D0FD074604E09E
:10205000FFF7CCFDC01B0228AED828688007F7D454
:102060002078000723D5E0690028686A0FD0304344
:102070006862FFF7BBFD074605E00AE1FFF7B6FD22
:10208000C01B022898D8686A8007F7D50FE040087F
:1020900040006862FFF7AAFD074605E0A4E0FFF7ED
:1020A000A5FDC01B022887D8686A8007F7D420786E
:1020B00004274007002860DA00200190E869C0008A
:1020C00008D4E869B9060843E861E8690840009067
:1020D0000120019071480168C90511D40168821579
:1020E00011430160FFF782FD009005E0FFF77EFDE0
:1020F0000099401A642877D868480068C005F5D56B
:10210000A06801280AD0002801D0052810D0286A2C
:10211000400840002862286AB84301E0286A30433A
:102120002862A068002812D0FFF760FD00900AE046
:10213000286A38432862F1E7FFF758FD0099411AF1
:102140005748814250D8286A8007F5D50DE0FFF73F
:102150004DFD009006E0FFF749FD0099411A5048F7
:10216000814241D8286A8007F5D40198002804D01C
:10217000E869012109078843E8612078C0063CD559
:10218000606901280CD0401D686B23D03843686318
:10219000686B400840006863FFF728FD064629E0A9
:1021A000686B38436863686B30436863FFF71EFDF4
:1021B000064604E0FFF71AFD801B022862D8686B10
:1021C0008007F7D5686BF8218843A169C9000843E7
:1021D000686312E0B8436863696BF8208143A069C3
:1021E000C0000143696308E04CE0FFF7FFFC801B7F
:1021F000022847D8686B8007F7D4206A002846D0A9
:1022000069680907890F022943D001273F06022880
:10221000286805D0B8432860FFF7E8FC044633E09F
:10222000B8432860FFF7E2FC064604E0FFF7DEFC57
:10223000801B022826D828688001F7D4E86AE16A62
:10224000000900010843E862616AA06A08436968FE
:102250007B22D20391430843686028683843286092
:10226000FFF7C4FC044604E0FFF7C0FC001B022893
:1022700008D828688001F7D509E0FFF7B7FC001BF4
:10228000022801D90320FEBD28688001F5D4002072
:10229000FEBD0120FEBD00000010024000700040A5
:1022A00088130000042204490428086902D09043DE
:1022B000086170471043FBE700E000E01548016843
:1022C0006431016014480168491C016013490868C1
:1022D000401C08601249134AC868401CC8609042FC
:1022E00016DB0020C8601048816D491C8165016DB6
:1022F000491C0165416D491C41650C49088B00284A
:1023000006D0401E80B20883782801D9782008833F
:1023100070470000900100208C0100200C0100207B
:10232000B00100201027000044190020781B002075
:10233000094910B5401E884201D9012010BD074C43
:1023400060610321081F02F043F80020A06107200C
:102350002061002010BD0000FFFFFF0000E000E052
:1023600010B5FFF7ABFF10BDFEE7000010B5002170
:102370000F4A0846516043009B18401C1981FF28F2
:10238000F9DD002005230B4ADB014400A418E41802
:10239000401CA1821028F8DB00200923DB01440047
:1023A000A418E418401CA186FF28F8DD002010BD09
:1023B0003C110020C413002010B5402802DB00208F
:1023C000C04310BD10221143C200094B4000D21877
:1023D000C01858240D23A1529B010021C3189986CF
:1023E000E300C0188186034800685065084610BDA8
:1023F000C4130020E007002070B504461E463830A4
:10240000049D04F0EDF820462A463146583004F089
:10241000E7F8002070BD000070B5104D064601467B
:102420002846FEF779FE0E4CE062FFF741FD294693
:10243000FEF75CFE60620B48314600680546FEF719
:1024400055FEA0622A46002307480F21FEF778FEBA
:102450002080E06A64302062002070BD40420F009E
:1024600070010020DC07002000004042F8B572B681
:10247000012212030921C9068A6200BF00BF00BF02
:1024800000BF8A61C117490F0818C0108446002098
:10249000104E0346009017E008200E4C00228021C9
:1024A0008502103C37687F0400D50A43A5624908BD
:1024B00000BF00BF00BF00BF00BFA561401EF1D13B
:1024C000D0436946C8545B1C6345E5DB62B600989F
:1024D000F8BD000010040048034610B50020024675
:1024E00002E09C5C6040521C8A42FADB10BD000096
:1024F000F8B508460D460978552901D0252903D09D
:10250000012A01DD451C521E344F602479792B7855
:102510006143334C0919334C252B30D0A3685B1C25
:10252000A360CB695B1CCB61B97800290FD0F97827
:1025300000290FD001292C4913D007231B02C918E9
:102540000A7501462948FEF732FE0020F870002087
:10255000C043F8BD2549264B55390A750146224826
:1025600007E037235B01C9180A750146204B1E4856
:102570002033C018FEF71BFEF878401CE6E76E79A2
:10258000802E06DDE068401CE060086A401C08629E
:10259000DDE7334608339A4208D2086A401C0862D5
:1025A000E068401CE0600220C043F8BDB11DFFF7A9
:1025B00093FFA919897981420DD02069401C2061BF
:1025C00079796020414306480818416A491C4162F4
:1025D0000320C043F8BD0020F8BD0000F00000203B
:1025E0002C0C0020F8090020C4130020D91A002068
:1025F000D5060000F8B50E4604462520069F079D27
:10260000089920706270A670E37027712F46002031
:1026100008376619372B1AD009DC1A46303A1300EE
:1026200003F002FD07261515262626172600612B26
:102630000DD006DC382B0AD0412B08D0422B17D105
:1026400005E0622B03D0632B01D0642B10D16571A0
:1026500002E06571002D03D02A46A01DFEF7A7FDFC
:10266000A91D2046FFF738FFB0710D20F0713846E4
:10267000F8BD0000F1B584B0FFF7B8FA0546FFF7E2
:10268000E7F9604E0446F079002806D0307A002839
:1026900003D0F068201A322805D8F0687D21201A6E
:1026A000C90088427ED9307A574A00281DD07179F6
:1026B00060235943554B0120585064205064707971
:1026C000401CC0B27071F17A884208D9B06AB46215
:1026D000201AF062B079401CB071012070714C4832
:1026E000008A4C4F002830D038E0706A401C70627D
:1026F00049484168491C4160717960200B46434359
:1027000042489C46181803695B1C036143695B1CC3
:102710004361F779002F02D1876A7F1C876287693E
:10272000BB4200D983613948032BC8D900236746CF
:10273000C351C8209064394843544800384941186F
:102740000F20800108188386B9E7FFF70FF9354994
:1027500080B28882C1B2F982000A38832F49B87DDD
:1027600010314870387E887072792F488B5C037006
:10277000891849784170602113464B43234900274B
:10278000C9588170C77005712B0A43712B0C837176
:102790002B0EC371F4606C462378B4799B089B00C0
:1027A000A40700E028E0A40F23436C46237000290F
:1027B00025D0EF210B402370029008211748009389
:1027C0000191412300212030FFF714FF13490246F5
:1027D0002031049802F046FC7179602041430B4897
:1027E00008184168491C4160C268F1688A1A42634E
:1027F000C1607563F7713772002005B0F0BD10211C
:102800000B43D8E7F0000020441900202C0C0020D6
:10281000781B0020C4170020F80900200C0B0020B2
:10282000C4130020041600202C0F0020F7B50878F0
:1028300086B00C46552801D0252802D0012A00DD9B
:102840004C1C4C4D627968796021049048434A4998
:102850002B4640188168491C8160474980390391A3
:102860001F6BDB68E678FF1A2B46A1789B69303E28
:102870000093330003F0D8FB13420B174242422966
:10288000424242424242424242422C4542003B487E
:10289000A37943542179A01D322301920091029023
:1028A0000021049A22E06F61009A974200DDAF6137
:1028B000324AA37953540021C7624161016BB94286
:1028C00000D207630120287218E00120E87115E0AA
:1028D0002A48A179017010300078A0712179A01DDB
:1028E0000192009102904223297900220398FFF778
:1028F00081FE02460399069802F0B4FB002009B05D
:10290000F0BD6F610098874200DDAF611B4AA0797E
:1029100050541B4A490089180F2292018918888651
:102920001848008A002809D11748C18E008F00027C
:102930000818164980B2888602F048F96A79602042
:1029400042430D480021161871616869F062316BCD
:10295000814200D230632046677A0A30FEF74BFC92
:10296000617B0002000A09060843B90071188863F8
:10297000A8E70000F00000202C0C00200C0B002029
:10298000C4130020781B00208417002004160020A8
:10299000F7B515460C46FFF75BF81A4E3063217801
:1029A0000020552903D1012D01DD641C6D1E3178F5
:1029B00000290FD00127F7712A4621460098FFF71A
:1029C00097FD002805D137722A4621460098FFF767
:1029D0002DFFFEBD71780029FBD00B4E2A46B06B4F
:1029E0002146401CB063009800F012F80028F0D196
:1029F00006482A46406C30652146009800F080F871
:102A0000FEBD0000F00000202C0C00204419002026
:102A1000F0B508460D460978552901D0252903D07F
:102A2000012A01DD451C521E297800231A4FDB4381
:102A30001A4C252906D0A068401CA060386C401CA8
:102A4000386409E014496E79896C491C802E05DDD3
:102A5000E068401CE060B9641846F0BD33460833B6
:102A60009A4206D2B964E068401CE0600220C0438C
:102A7000F0BDB11DFFF730FDA9198979814208D059
:102A80002069401C2061F86C401CF8640320C0439E
:102A9000F0BD0020F0BD00002C0C0020F809002043
:102AA000F8B5FEF7D5FF134B1A69197900291FD025
:102AB0005C7A1149002C05D07D20800148640020FB
:102AC000587215E00C4E0D4C851A8036A54204D97B
:102AD0007D2292018A64012206E01219904207D9F0
:102AE0007D2292018A6402228A67C8671869306071
:102AF0000020F8BDF000002044190020E02E000066
:102B0000F7B5087884B00C46552802D1012A00DDBB
:102B10004C1C5B480168491C016065796078594923
:102B2000594A0391574E11798036884208D0FF28C0
:102B300006D0706C401C70640020C04307B0F0BD2C
:102B4000884201D0FF287DD1106B009010610120D8
:102B500050724C4FE078A03F372873D007DC3038F4
:102B6000030003F061FA068B138B8B8B238B612898
:102B700068D004DC382865D041287FD11FE0622866
:102B80007CD063287AD0642878D16CE0A079387042
:102B90003C4890380078A071009810612279A01DFF
:102BA0003223009201950290002250E0002021790A
:102BB00036230091019002460290012147E0A0795E
:102BC0003870E179314B79705975E37AA17A1B023B
:102BD000CB182D49CB6101F0F9FF2B48877AFEF71E
:102BE000C5FE2849294A90390870203A527D4A701A
:102BF000A0714878E071B80067728019018FA172E6
:102C0000018F090AE172816B090C2173806B1E49E7
:102C1000000E60731C48807A401CC0B288720A287B
:102C200001D300208872207969460870C00603D558
:102C30007D20174980018864A01D2179422300224C
:102C4000019500E01AE002900F4800910179039885
:102C5000FFF7D0FC0246F06B401CF0630399049828
:102C600002F000FA0AE0E179A07909024018217A1D
:102C7000637A09041B06C9184018D06100205DE77B
:102C8000F8090020AC0B0020F000002024160020E2
:102C900044190020034610B50020024602E09C5C67
:102CA0006040521C8A42FADB10BD30B50D46084622
:102CB00009781446252901D0012030BD062C01D207
:102CC000032030BD611EFFF7E5FF29192039C97FB8
:102CD000814201D0042030BD002030BDF8B51E4631
:102CE0000B465527069D0799077043708270C67082
:102CF000044605712A46401DFEF759FA691D204613
:102D0000FFF7C8FF014660194171A81D052E02DAC0
:102D1000002E00D10020F8BDFEB516460F46054630
:102D2000FFF7C3FF040014D068460472042000902B
:102D300002A90B4801910278401E0178EE23094850
:102D4000FFF7CCFF02460749284602F08BF92046E0
:102D5000FEBD32463946284600F006F8FEBD0000AA
:102D60002D010020BC0F0020F7B5FA4886B04F783F
:102D700042688260421C15788E782D0936072D0135
:102D8000360F0B7935431570F34A029200780C46E2
:102D90000490874201D0FF2F77D12146E678093190
:102DA000EE488C46332E72D028DCED49182E0A6886
:102DB0006CD012DC072E20D008DC002E65D0012E4E
:102DC0003ED0032E41D0052E7ED160E0112E7CD066
:102DD000162E7BD0172EF7D13FE2232EEED006DC45
:102DE000192E74D0212E73D0222EEDD18FE1242EF6
:102DF000E4D0312E4BD0322EE6D1BFE0582E68D031
:102E000012DC542E66D008DC342E71D04F2E70D0D8
:102E1000502E6FD0532ED7D16EE2552E6BD0562E3A
:102E20006AD0572ED0D164E23046633804210300C3
:102E300003F0FAF809F0EFEE171D4A104A154A00A0
:102E4000641D00930194012351E2C649182003E058
:102E50003946C7E2C4490C200191009005E0C348FF
:102E6000F6E1C24910395020F6E733463FE2E179F6
:102E70000020B94A03E023185B7A1354401C8842AF
:102E8000F9DBB54802F07AFEA3E075E2EEE1A27943
:102E9000617912028918E27989B2882B2DD0892BA9
:102EA0002FD08A2B31D0832B34D0842B37D0852B55
:102EB0003AD0862B3DD0872B40D08B2B43D08C2B08
:102EC00046D0FE2B1DD006E097E29FE1AEE1EDE19A
:102ED000C9E066E227E2A92B3FD0B32B41D0992B62
:102EE00042D0A12B45D09C481038401800925FE298
:102EF00044E0F6E1F1E140E249E2490009189C486A
:102F00003AE0490009189B4836E0490009189848FA
:102F1000203831E049000918952080002CE0490054
:102F200009189D20800027E049000918A52080008D
:102F300022E049000918FD2080001DE04900091821
:102F40008B48A03818E049000918DD20800013E004
:102F500049000918BD2080000EE049000918864884
:102F60000AE04900854807E0854849000818001D27
:102F7000BCE749000120C0060818B7E7A2796179CB
:102F800012028918E27989B2882B25D0892B27D0A3
:102F90008A2B29D0832B2CD0842B2FD0852B32D079
:102FA000862B38D0872B3BD08B2B3ED08C2B41D01F
:102FB000FE2B45D0A92B47D0B32B49D0992B4AD013
:102FC000A12B4BD064481038401800226146FEF710
:102FD000EEF80020009024E149000918644840E020
:102FE0004900091863483CE0490009186048203846
:102FF00037E0490009189520800032E0490009189F
:103000009D2080002DE049000918A520800028E0BF
:10301000DFE1D2E1CEE149000918FD20800020E087
:10302000490009185248A0381BE049000918DD2062
:10303000800003E049000918BD2080000818C4E79B
:10304000490009184B48F9E7490009184A48F5E7CB
:1030500049004A48F2E74900494802E04900012096
:10306000C0060818B2E7A27961791202891809220C
:10307000920189B2002B0FD0012B13D0022B1CD050
:10308000032B20D0042B26D0052B2AD0062B28D0AA
:10309000082B34D000202AE00B095B00181833E01D
:1030A000012024E00B095B00181811E00A07120F39
:1030B000012191400840F3D119E00A09520010188B
:1030C0000522D20120E00A09520010180F229201B5
:1030D0008018808EEAE70A09520010180122920235
:1030E00012E0C90008184030007E4006C00F694653
:1030F0000873012003A9212301910090F7E00A0938
:10310000520010180922D2018018808ACEE7A279D5
:1031100061791202891889B2002B33D0012B3AD081
:10312000022B41D0032B48D0042B4FD04022052B3B
:1031300054D0062B52D0072B5BD000206946087371
:1031400000200090034803A9401C0191027822232B
:103150007EE600002C010020BC0F0020C4130020DC
:103160003C1100204C6D0008ACF7FF1F107C0008DC
:10317000B4040000B4050000B40600002C0C0020CC
:10318000441300200B070909490009181B0F95205B
:10319000E279800035E00B070909490009181B0F87
:1031A0009D20E27980002CE00B07090949000918ED
:1031B0001B0FA520E279800023E00B0709094900D5
:1031C00009181B0FFD20E27980001AE00B0709099E
:1031D0001B0F49000918E2798D4812E0C900081850
:1031E0004030018B9143E279D207520E11430183A3
:1031F000A6E70B070909490009188548E2791B0F62
:1032000080300818194601F051FF99E7002B05D0CE
:10321000012B00D0DDE602F007F9DAE602F03CF916
:10322000D7E601907B48E378027811E6A1796079CE
:1032300009024018E179784A80B2002B0AD0774C15
:10324000012B03D0764B9B8A002B03D04000001942
:103250000091ADE040008018FAE7002A01D000207C
:103260000860002000901723019040E0002A01D060
:1032700000200860A17960790902401885B2E279DE
:103280000020684903E02618767A0E54401C9042CC
:10329000F9DB6449284602F07FFC002009340090E5
:1032A00001905C48039402781823D1E5A1796079F4
:1032B000090241185A48C182818A00290BD0002195
:1032C0008182574801F08EFE002000900190514805
:1032D00019230278BCE50121F2E75148038300205D
:1032E00002E04F490020088300900190E3782A46CD
:1032F000AEE54B492020AFE5A1796079090240187D
:10330000494980B20A18E179121D782801D30021B9
:1033100005E00B18782B02D97821081A81B2C8B2BF
:1033200001920090A1E5A1796079090240183E4917
:1033300080B20B18E2791B1D782801D3002205E02A
:103340001118782902D97821081A82B261461846E4
:10335000FDF72DFF0020009001902E48E3780278C1
:1033600039460298FFF7BAFC02460299069801F026
:1033700079FE2D4802F030FC3CE02B4802F02CFC9A
:1033800000200090019023485523027860E52448EE
:1033900001F028FE0020009001901E48562302787C
:1033A00056E5032109022148FDF71AFF002000908D
:1033B00001905AE51E481F4A4DE7A179607909023C
:1033C0004018E17980B20D01FEF7BEFAE9B2009132
:1033D00027E7FEF7E5F80020009001900D486523EF
:1033E000027835E50298FFF779FC024602990698C3
:1033F00001F038FE002009B0F0BD022069460873D4
:1034000003A901200191EE232A4600900499E9E7DF
:10341000140400002D0100200080000800A0000816
:10342000781B0020BC0F0020441300202C0C00202F
:10343000C4130020F405000070B5FEF77BF81648B1
:1034400000F078FA154D164C6869A065124881683D
:1034500061658188491C81808088E0640E4801F0A4
:10346000C1FD2868206768686067A868A0670122B6
:103470000C4B1146A06DFEF701F820468030E9683C
:103480000160A9694160E96981602969C160296AAF
:103490000161002070BD0000781B00204001002069
:1034A000441900203930000030B5836801221340F0
:1034B00002D00022104630BD8C684B68C968234397
:1034C000C468034D2C4021430B43C360F2E7000066
:1034D000C73FFFFF30B583680122134002D00022AE
:1034E000104630BD18C94D6823430C6889682C43C9
:1034F00023430B43C168024C21400B43C360EFE7F9
:103500003CC2FEFF08B504494A6902434A61496961
:103510000140009108BD00000010024008B50449B8
:10352000CA690243CA61C9690140009108BD00002F
:103530000010024008B504498A6902438A6189691A
:103540000140009108BD00000010024070B5094E16
:1035500004467618203E049D0C34F17F0830102D6F
:1035600003D00A50F07F035170BD0A51F17F0B5018
:1035700070BD0000F46D0008044A51182039C97F5D
:10358000425852085200425070470000F46D000843
:10359000044A51182039C97F425801231A43425026
:1035A00070470000F46D0008044A51182039C97FA3
:1035B000425802231A43425070470000F46D00083D
:1035C000054B10B559182039C97F435803242403EB
:1035D000A3431343435010BDFA710008054B59181B
:1035E0002039C97F001D0B581B0C1B0413430B50C3
:1035F00070470000F46D0008054B10B559182039CC
:10360000C97F4358034C23401343435010BD00006F
:10361000FA710008EFBFFFFF054B10B559182039AC
:10362000C97F43588024A3431343435010BD000077
:10363000FA710008054B10B559182039C97F435855
:103640000324A402A3431343435010BDFA7100089E
:10365000054B10B559182039C97F43582024A3437E
:103660001343435010BD0000FA710008054B10B51C
:1036700059182039C97F43584024A343134343506A
:1036800010BD0000FA710008054B10B5591820391B
:10369000C97F435803242402A3431343435010BD5E
:1036A000FA710008F0B500233CE001249C40224060
:1036B00037D04F6806681446544365006519AE4319
:1036C00067433E4306604E68012E01D0022E05D1AD
:1036D0008F6886686743AE433E4386600F69C6685D
:1036E000AE4325467D432E43C6604D68022D18D15A
:1036F0004D69FF2A09D8066A544354432201121B1C
:1037000096436C43264306620BE0140A224662434A
:10371000624362431401A61A446A6A43B4431443E1
:1037200044625B1C0A681446DC40BED14A68012A28
:1037300001D0022A06D10A68C968436893434A4304
:10374000134343600120F0BD10B5044601F07EFA3A
:10375000206001F061FA606001F06CFAA06010BDB9
:10376000014610B5002000290FD1104A116B8907BE
:10377000890F01290AD0022911D0032909D001F0AB
:1037800065FA01F049FA01F055FA10BD01F05EFA50
:1037900010BD11688907C90FFAD0054810BD116A1C
:1037A0008907C90FFAD00120C00310BD00100240E4
:1037B00000127A00F0B50268194B1A4C984201D0F9
:1037C000A04203D17025AA434D682A43164D174ED7
:1037D000174F98420AD0A04208D0164CA04205D0FC
:1037E000A84203D0B04201D0B84204D1032424023D
:1037F000A243CC68224302608A68C2620A8882625D
:10380000984205D0A84203D0B04201D0B84201D1BD
:10381000097C016341690122114341611046F0BDF9
:10382000002C0140000400400040014000440140E1
:10383000004801400020004041680122D20291432B
:10384000416081680822914381607047FEB504465B
:1038500000680D460026C007C00F4FD1E9686868B0
:10386000AA6908432969114308432168244A114081
:1038700008432060A8686168032212039143014352
:1038800061606869A168121191430143A1601D48FC
:10389000844203D10020FFF763FF12E01A488442FC
:1038A0000BD01A48844208D01948844205D01948E0
:1038B000844202D01848844220D16846FFF744FF72
:1038C000029800281AD02968002917D00126AA6971
:1038D000F3039A420CD140004A088018FDF706FC19
:1038E0000E4980B201400007420F0A43E26005E042
:1038F0004A081018FDF7FAFB80B2E0603046FEBDC2
:10390000F369FFEF003801400044004000480040E8
:10391000004C00400050004000140140F0FF000047
:1039200010B580220249FDF742FC002010BD0000C6
:10393000646D0008F0B5154A00215514144C154F5C
:103940000CE0D65ABE4208D19B185B886668B34229
:1039500003D90AC44B1C2360083C491C4B01AB42F1
:10396000EFD321680123002905DB490189182022B2
:1039700001F006FA00E08380A06840012030A842F0
:1039800001D90020A0600020F0BD000000C80008A0
:1039900040010020AA5500001FB50B46024604A1B5
:1039A000684602F02DFB0146684601F013F91FBD81
:1039B000201B5B25643B25644800000070B5012096
:1039C0008AB04002FFF7B6FD224CA06A03263043BE
:1039D000A0622149B0050A68824302430A60A26AD4
:1039E00083111A43A2620A68824302430A600025D7
:1039F00005950695079505A920460895FFF754FDFE
:103A00000120039000950195029569460495204692
:103A1000FFF760FDE16804208143E1606169C90846
:103A2000C9003143616161680143616060680821D8
:103A300088436060A06817218843C9070843A060D5
:103A4000A068C00FFCD1A06804490840401CA060D9
:103A50000AB070BD0024014008270140E8FFFF7F45
:103A600010B50120FFF74EFD00210A2000F08EFC6A
:103A70000A2000F081FC00210B2000F087FC0B20C5
:103A800000F07AFC10BD0000F0B5012087B04004C2
:103A9000FFF738FD01208004FFF734FD0120C0044A
:103AA000FFF730FD01208005FFF72CFD1C480125A4
:103AB000002403266A46049551C20927FF06694679
:103AC0003846FFF7EFFD1920000203946A4604947C
:103AD00061C269463846FFF7E5FD2802B861114822
:103AE0006A46049551C2104F69463846FFF7DAFD21
:103AF0000B20000303946A46049461C26946384669
:103B0000FFF7D0FD0720400300900294039469461C
:103B1000019504940548FFF7C5FD07B0F0BD00000E
:103B2000C0800000E743000000040048000800488F
:103B30000848074901600849016004214160074ABB
:103B40008260C1684907FCD1026105490160704784
:103B5000CCCC00000030004055550000FF0F0000A5
:103B6000AAAA000010B586B014216846FDF738FBFC
:103B70001020FFF7D3FC0021112000F007FC1120DA
:103B800000F0FAFB2F2069460880002001900848C9
:103B9000084C02902046FFF70DFE206880218843E4
:103BA0002060E06801210843E06006B010BD00001D
:103BB000E70300000010004070B501208EB08003C4
:103BC000FFF7B8FC03204002079002200890032072
:103BD00000240990012509200A9407A90C950B944B
:103BE000C006FFF75FFD3A4E102202213046FFF774
:103BF00003FD002202213046FFF7E2FC00220221F1
:103C00003046FFF725FD002202213046FFF72EFD4A
:103C1000802202213046FFF7FFFC002202213046BD
:103C2000FFF732FD002202213046FFF703FD00229C
:103C300003213046FFF7E0FC002203213046FFF766
:103C4000BFFC002203213046FFF702FD00220321C2
:103C50003046FFF70BFD802203213046FFF7DCFCE6
:103C6000002203213046FFF70FFD002203213046DA
:103C7000FFF7E0FC00211B2000F088FB1B2000F078
:103C80007BFB1448694600680090019402940394F9
:103C9000059406940C20104C04902046FFF7D6FDA6
:103CA0006068290508436060606849000322520586
:103CB000904308436060A06849120843A060204612
:103CC000FFF7BAFD2068284320600EB070BD0000E9
:103CD00000000240D800002000380140F0B58DB04F
:103CE0001C2106A8FDF77CFA18216846FDF778FA32
:103CF000012464042046FFF711FC2046FFF702FC74
:103D0000012500240E200226032703956A46059507
:103D10000494C1C209206946C006FFF7C3FC00969F
:103D20000920039504956946C006029701960595FA
:103D3000FFF7B8FC464E102204213046FFF75CFC2A
:103D4000002204213046FFF73BFC002204213046CC
:103D5000FFF77EFC002204213046FFF787FC80221B
:103D600004213046FFF758FC002204213046FFF7BB
:103D70008BFC002204213046FFF75CFC0022052169
:103D80003046FFF739FC002205213046FFF718FCCA
:103D9000002205213046FFF75BFC0022052130465A
:103DA000FFF764FC802205213046FFF735FC002236
:103DB00005213046FFF768FC002205213046FFF759
:103DC00039FC00211C2000F0E1FA1C2000F0D4FA9C
:103DD000A61EFF21304600F0D9FA304600F0CCFA9A
:103DE0001C48EE03006806900794089409940C2080
:103DF0000AAA51C2184C06A92046FFF727FDA06861
:103E000021140843A060A068B0433043A06020683C
:103E10001F214905884308432060206849118843D1
:103E200008432060606829050843606060684900B5
:103E30007A05904308436060A06849120843A06077
:103E40002046FFF7F9FC2068284320600DB0F0BD44
:103E500000000240DC0000200044004010B58EB09D
:103E60001C216846FDF7BCF9182107A8FDF7B8F931
:103E70000124A4042046FFF751FB2046FFF742FB34
:103E800018200790022008900320099000240420A5
:103E90000C900A940B9407A91348FFF703FC002128
:103EA0001D2000F073FA1D2000F066FAE120800268
:103EB00000900C2004900194029403940594012036
:103EC000C0030A4C069069462046FFF7BFFCA06875
:103ED000A1140843A0602046FFF7AEFC2068012132
:103EE000084320600EB010BD0004004800480040A8
:103EF00010B58EB01C216846FDF772F9182107A88D
:103F0000FDF76EF901200005FFF708FB0120800492
:103F1000FFF7F8FA18200790022008900320099074
:103F2000002404200C900A940B9407A91348FFF76F
:103F3000B9FB00211D2000F029FA1D2000F01CFA19
:103F4000E120800200900C200490019402940394DC
:103F500005940120C0030A4C069069462046FFF7ED
:103F600075FCA068A1140843A0602046FFF764FC1C
:103F700020680121084320600EB010BD00040048F5
:103F80000050004030B58DB01C216846FDF728F97F
:103F9000182107A8FDF724F92020FFF7CBFA01200C
:103FA0004004FFF7AFFA302007900220089003206A
:103FB0000990052000240C9009200A940B9407A96D
:103FC000C006FFF76FFB00211D2000F0DFF91D2068
:103FD00000F0D2F9E1200002009001250194029442
:103FE00003940C20ED0304AA31C20B4C6946204611
:103FF000FFF72CFC6068A84328436060A068A11408
:104000000843A0602046FFF717FC20680121084301
:1040100020600DB030BD00000014014000B508461E
:10402000042A02D80020C04300BD01787F2902D9AC
:104030000120C04300BD41784906490E1F2902D91D
:104040000220C04300BD114602F094FA0028F9D0C6
:10405000042000BDF7B588B00F460A9A0898FFF70C
:10406000DDFF0690002803D00020C0430BB0F0BD58
:10407000BD483A7800783946824273D18C784A78C4
:10408000CB78B98824024DBAB8491C4308704A70ED
:1040900001200790200521070226000E090F1300BA
:1040A00001F0C2FF11A60A508DA7BFDDA6A6A6A6E5
:1040B000A6A6A6A6E9F0A600E81DC008AB49039095
:1040C0008870002038E000270120059701900098B3
:1040D000C000049026E0210701222009090FD20226
:1040E000944207D24200A2481218092080011018F9
:1040F000808E05E042009E481018FF308130808A93
:10410000FDF798FB002801D0019807430198641C33
:104110004006000E01900598A4B2401C05900828A6
:1041200004DA049805994018A842D4DB8F48009916
:104130004018C7700098401C039900908842C2DB69
:10414000761854E0E81DC008884903908870002064
:1041500030E0002000900120019002980027C0006C
:1041600004901DE0FDE02005000E4200804821077C
:104170001218092080011018090F808AFDF75AFBD8
:10418000002803D001990098084300900198641C0E
:104190004006000E7F1CA4B20190082F03DA049899
:1041A000C019A842DFDB7149029A00988918C870CB
:1041B0000298401C039902908842CADBC0E768005D
:1041C0006A498446887000200EE021184A00684938
:1041D000470052180921C9015118898E634A0B0AF8
:1041E000BA18D3701171401CA842EEDB17E0761CA0
:1041F0008DE068005D4A8446907000200DE0211833
:104200004B005B4947005B18092189015918898ACD
:10421000BF180B0AFB703971401CA842EFDB6644E3
:10422000E5E7002D12D0FF221202954207D142008D
:104230004F4812189D208000101800F02FFF3946BB
:104240004A480A9AFCF7B3FF0A9E85E042004848B4
:1042500012189D208000101800F0E0FDEFE738797B
:104260007979000208434249620052180921C901C4
:1042700051188886E3E7E81DC0083C490390887020
:10428000002036E047E03818C07900900120019006
:10429000002005900298C000049024E0210701222C
:1042A0002009090FD2029442009B019A07D21A40BA
:1042B00043002F481B189D208000181805E01A4065
:1042C00043002B481818FF30953000F0FBFE019892
:1042D000641C4006000E01900598A4B2401C059095
:1042E000082804DA049805994018A842D6DB0298F9
:1042F000401C039902908842C5DB1C48B978817044
:10430000F978C1703979017179794171361D069852
:10431000002814D025E000200EE04100C919CA7918
:10432000097A12020A4321184B0011495B1809212E
:10433000C90159188A86401CA842EEDBDDE70798C0
:10434000002809D0B1B2094802F014F9074988558C
:10435000000A89194870B61C32460449089800F0D2
:1043600081FE002082E6000038010020BC10002001
:10437000C413002070470000C106C90E0120884008
:10438000014908607047000000E100E08307FF2258
:10439000DB0E9A408907090E994000280BDA0007C6
:1043A000000F0838830808489B001818C369934316
:1043B0000B43C3617047830804489B0018180368C7
:1043C00093430B430360704700ED00E000E400E01E
:1043D0008307FF22DB0E9A408907090E99400028C7
:1043E0000BDA0007000F0838830808489B001818EC
:1043F000C36993430B43C3617047830804489B0020
:104400001818036893430B430360704700ED00E006
:1044100000E400E070B572B60125094A2D039561EC
:1044200080210C028B019362084201D0946100E06C
:10443000946249089361F6D19562956162B670BD48
:104440000004004810B501200449C0064860044833
:104450000168491C016000F005F810BD00ED00E0A6
:10446000D400002070B5094DE86F00280CD0084C2E
:10447000084902202268FEF78BFA00202060E867D6
:104480008021044801F086FA70BD00007809002000
:10449000E40000208C0A002010B50648054B007887
:1044A0000021403B5A1840325478491C14700F299F
:1044B000F8DB10BD0414002010B5084C084B012295
:1044C0000221A06DFCF7DAFF064800F08BFDE06DDD
:1044D000401CE065A06D2066002010BD441900203E
:1044E00039300000781B00200248C16D491CC165AD
:1044F0000020704744190020F3B5FA4D85B02868B4
:1045000000286FD0686800281CD000220D210820E8
:1045100000F0EEFD00221146082000F0E9FD012226
:104520001146082000F0E4FD00200146EE4A131871
:104530004033401C19701028F8DB00260121144676
:1045400040347BE20122E1E7B2000598059B805CE4
:10455000D7187A78019201257B8800931B2873D0A5
:1045600012DC0246030001F05FFD1B5C7272727286
:1045700072723E3E3E3E3E3E5C5C5CA7A7A73E3E5E
:10458000BEBEBEBEBEBE5C00342870D011DC01468B
:104590001C390B0001F048FD18A7A7A7A7A7A7A7DC
:1045A000A7A7A7A745454545454545454545454533
:1045B000F7453A2873D008DC014635390B0001F085
:1045C00033FD05E26E56E26E3000DC2804D004DCD8
:1045D0003B28EFD0C82824D120E1DD28FCD0FA28E0
:1045E000F9D11BE133E2D01F030001F01DFD0E08DD
:1045F0000A10181B1D1A1A1A1A1A1A20261A207CB9
:104600004AE0FFF749FF00281FD0207C3AE0FFF77F
:1046100043FF002816D1207C002813D125E000F0AC
:10462000C3FAF5E12078F7E7FFF736FF1DE0207CBD
:1046300000280AD0002905D007E0207C002804D1FA
:10464000002902D0012010E04DE000200DE0130011
:1046500001F0EAFC070C050E111B262E0C0000F0E1
:10466000A3FA00990198FDF7F9F82074D0E11AE156
:1046700000F09AFA0CE0207C0028E6D0009901981E
:10468000FDF7ECF80028E0D0DCE7207C0028DCD047
:1046900000990198FDF7E2F80028D6D1D2E758E159
:1046A000207C0028CED100990198FDF7D7F8B3E718
:1046B000207C0028ECD0C5E7102804D0112804D0B5
:1046C000122AAED10AE0227C03E0207C0028A8D088
:1046D00001220099019800F00BFD99E1207C00284F
:1046E0009FD00022F5E715383D79030001F09CFCCE
:1046F000120A1215181B0F1E3C4C5B6A2D7981851E
:10470000898D7D9400F050FA13E0207484E000F06D
:104710004BFA1DE000F048FA29E000F045FA36E0D7
:1047200000F042FA42E000F03FFA4EE0207C002820
:1047300070D028460099FDF71FF90546F988787969
:10474000FDF71AF9854263D064E0207C002861D02F
:1047500028460099FDF710F90546F9887879FDF7A4
:104760000BF9854254D155E0207C002852D02846D0
:104770000099FDF701F90546F9887879FDF7FCF80D
:10478000854245DB46E0B1E0207C002842D0284647
:104790000099FDF7F1F80546F9887879FDF7ECF80E
:1047A000854235DC36E0207C002833D0284600994D
:1047B000FDF7E2F80546F9887879FDF7DDF88542DE
:1047C00026DD27E0207C002824D028460099FDF72C
:1047D000D3F80546F9887879FDF7CEF8854217DADF
:1047E00018E0207C002813D1A3E7207C00280FD1FB
:1047F000AEE7207C00280BD1B9E7207C002807D148
:10480000C5E7207C002803D1D0E7207C0028DCD03D
:1048100001207AE7002078E70225F9E03F79154684
:10482000C8280DD0DC2823D0DD282AD0FA28F3D1DF
:104830002D48E90008184030007EC0062AD508E05F
:104840002948E90008184030007EC00601D4002144
:1048500021E0207C002822D038460099FDF78CF812
:104860000146284600F0E2FA284600F0F5F84CE749
:104870001D48E90008184030007EC006E9D4012137
:1048800009E01948E90008184030007EC006E0D46D
:10489000022100E003212846FDF78EFDD9E72846D6
:1048A00000F01AFEE0E73F790225342802D03728CD
:1048B00016D108E0207C002812D038460099FDF778
:1048C0005BF8401C07E0207C002809D0384600999E
:1048D000FDF752F8401E02463846009900F07EFC73
:1048E00096E000003C110020C41300203D79797946
:1048F0000291F9880191332814D035281BD038282B
:104900008AD1207C002887D00298FDF735F8074629
:1049100028460099FDF730F83A1A0199029800F0FC
:104920005DFC79E7207C0028FBD028460099FDF744
:1049300023F80246F1E7207C0028F2D028460099AF
:10494000FDF71AF8054601990298FDF715F82A189F
:10495000E3E73A7979790291F9880191797A0391BB
:104960007D89362806D0392812D03A281FD03B2816
:104970004DD131E0207C002849D010460099FCF749
:10498000FBFF074601990298FCF7F6FF3A180CE086
:10499000207C00283BD010460099FCF7EDFF07462D
:1049A00001990298FCF7E8FF3A1A29462CE0207C8E
:1049B00000282CD010460099FCF7DEFF07B20199C1
:1049C0000298FCF7D9FF00B247433A4629460398BC
:1049D00000F004FC3A1416E0207C002817D01046A2
:1049E0000099FCF7C9FF07B201990298FCF7C4FFD0
:1049F00001B23846FCF790FB02B20F4629460398F5
:104A000000F0ECFB3A46691C039800F0E7FB032535
:104A1000301141000F48012308183107090F02899E
:104A20008B401946114000D00121277C0830002F0F
:104A300001D01A4300E09A43028076190698864214
:104A400000DA81E503494868401C4860002007B04F
:104A5000F0BD00003C110020FEB50746402802DBF7
:104A60000020C043FEBD2C48F9000E1800964036C9
:104A7000348BE10601D40020FEBDA1063CD56106C1
:104A80003FD42649096800980A25406D0190081A0C
:104A9000A1070FD0A107890F012905D0022905D050
:104AA000E143890705D005E0642503E07D25ED009D
:104AB00000E01B4DA84224DB2946FCF72DFB0146F4
:104AC00015487A0012180B20800110188446808E39
:104AD000019B401869435B18009980B24B650D211A
:104AE00089015118898E814203D8084640210C4320
:104AF00034836146888604E0600602D54020844302
:104B00003483307EB9B24006C20F052000F0F0FABF
:104B1000307E4006C00FFEBDC4130020E007002019
:104B200010270000F7B50446FCF7FBFE0546029986
:104B30002068A942A16806DC4018029A0199FCF796
:104B400036FB029919E040182A460199FCF72FFB21
:104B500029462046FCF7D8FC2046FCF7E2FE064634
:104B60000298471BB7420DDCA16820683A464018FE
:104B700001994919FCF71BFB39462046FCF7C4FC98
:104B80000298FEBD002E0CDDA16820683246401858
:104B900001994919FCF70BFB31462046FCF7B4FCA0
:104BA000AD192846FEBD0000074A0F2011183F230B
:104BB0005B5C4031401E0B700028F7DC024940313D
:104BC000087C087070470000C413002000B5FFF790
:104BD00021FC00BD10B50C460A4601460348FFF70C
:104BE000A1FF00F0BFFE204610BD00003C090020E0
:104BF00010B50C460A4601460348FFF793FF00F044
:104C0000B1FE204610BD00003C09002010B50C4646
:104C100000F010FF204610BD04494968F022114001
:104C2000034A0909515CC840704700000010024067
:104C30000472000803494968034A4905490F515C59
:104C4000C8407047001002401472000810B50748B1
:104C500041680C200140064805D0042904D00829E9
:104C600001D100F009F810BD024810BD001002404B
:104C700000127A00001BB70010B50D4C60680321CC
:104C8000C90301220840D203811A0A4802D0914286
:104C900000D10948E16A0907090F491CFCF726FA07
:104CA00061680F2292041140890C891C484310BD91
:104CB0000010024000127A00001BB7000920C00655
:104CC00000694106C90FC943C907CA0D012149023C
:104CD0008A430106C90FC943C907890D0A43012147
:104CE000C00B8902C043C0078A43400D02432248DB
:104CF00001690120C00282438807C00FC043C0077A
:104D0000000D02430120000382434807C00FC04347
:104D1000C007C00C024350088A06D30F012240008E
:104D20009A431043022290434A06D20FD243D2073D
:104D3000920F1043042290430A06D20FD243D207A7
:104D4000520F104308229043CA05D20FD243D20714
:104D5000120F8905C90F1043C9431022C907904398
:104D6000C90E0843054909695202C90BC943C9075D
:104D70009043890C0843704700040048000800482D
:104D800070B5D417A40F0023A418A51003E09C004D
:104D90000E5906515B1C9D42F9DCD40F6B00A41820
:104DA000651003E05C000E5B06535B1C9D42F9DC62
:104DB000104670BD00B5FFF781FF00BDF8B50023B8
:104DC00084468025DB431248002421462A464A4374
:104DD000121817880F4EB74209D17E26B75A0E4EC9
:104DE000B74204D15288A24201DD0B461446491C49
:104DF0000829EBDB082B06D26B431918802260468A
:104E0000FFF7BEFF02E06046FEF78AFD0020F8BD16
:104E100000C00008AA550000A55A00000B07028830
:104E20001B0F012199408A430280704730B540280A
:104E300002DB0020C04330BD0D4CC20013191A46DE
:104E40004032157EAD0611D4400000190D24A40196
:104E50000419A1860B240021A401001981860548AC
:104E600000685865108B202108431083002030BD56
:104E7000C4130020E0070020034610B500200246BE
:104E800004E09C5C2018521CC0B2D2B28A42F8D313
:104E900010BD000010B50B4C20461E388278611FF3
:104EA0004A704922227000796070085CA07003216A
:104EB0002046FFF7E1FFE0700421204600F040F8B3
:104EC00010BD0000F601002010B51C4C2078002811
:104ED00024D0207B80062DD1607901220023002878
:104EE00006D0A271E07900280AD0401EE07107E0E8
:104EF000A068401CA0600A2802D91420E071A371A8
:104F00006078002816D02179491CC9B221718142EC
:104F100000D922716371FFF7BDFF0BE02069401CCF
:104F20002061C82801D9642003E0E079002801D07D
:104F3000401EE071E068401CE06010BDD801002018
:104F400010B500F005FE10BD70B5044604291AD155
:104F50000321FFF791FFE178884214D1184900221C
:104F60000878002820780FD00B461433692808D120
:104F700065780879854204D101254D718A60A2784F
:104F80001A545878C87070BD4928FCD10C4D60780F
:104F90004B781E359842F6D1A078C87069200A6116
:104FA0002870487868708878A87003212846FFF731
:104FB00063FFE87004212846FFF7C2FF70BD0000C0
:104FC000D801002010B500F001F810BD0348816839
:104FD000C907C90F00D0C068704700000030014009
:104FE0007047000070B51A4C6168491C616019492E
:104FF0000180A18841801849CA6C8280496D816016
:10500000112181831549C183A1684A0114495118AE
:1050100000250B462A469E5CFF2E04D1521C202AF6
:10502000F9D3002D10D02022FCF758FBA068206097
:10503000401CA0604001012189022030884201D932
:105040000020A060002070BD202200F0FBFDEDE7F5
:1050500040010020AA55000044190020A55A000074
:1050600000C8000810B514460A46012802D00228DC
:1050700006D00DE021461046FFF7BAFD054804E0D2
:1050800021461046FFF7C2FD0348816F491C816726
:10509000204610BDE4080020780900200B07028894
:1050A0001B0F012199400A43028070470907090F2D
:1050B00001238B400188002A01D0194300E0994365
:1050C0000180704710B5002A02D0FFF7E7FF10BD3E
:1050D000FFF7A4FE10BD0907090F01238B400188CB
:1050E000002A01D0194300E0994301807047000075
:1050F00070B50B051B0E204C5B000D071C192D0F06
:10510000030000F091FF09060B14191E22272C3111
:105110003600FF292DD89520800003E0FF2928D8EC
:105120009D20800020182946FFF7D5FF21E0FF29A8
:105130001FD8A5208000F5E780291AD2FD20800025
:10514000F0E7802915D20D48ECE7402911D2AD20B7
:105150008000E7E740290CD2B5208000E2E78029F3
:1051600007D206482030DDE7802902D2034880308C
:10517000D8E7002070BD0000C41300201404000014
:105180000121C903034A002801D09162704791614F
:10519000704700000008004801218903034A0028E5
:1051A00001D091627047916170470000000800488B
:1051B00001210922C902D206002801D0916170475D
:1051C0009162704701214903034A002801D091628E
:1051D000704791617047000000080048F0B5304CFE
:1051E0004B001C190923DB01E6180B23DB01E51832
:1051F00092B28A283DD00EDC294F4B00DF190923DB
:105200009B01FF188338030000F00EFF0714181CE1
:1052100021262D46480099283ED006DC8B282CD02C
:105220008C2831D08D2839D133E0A12834D0FE2804
:1052300034D131E0102931DABA822FE010292DDA89
:10524000BA862BE0102929DA0520C00108E00829D8
:1052500024DA0F20800114E008291FDA01208002DF
:10526000201882821AE0802918DAB28616E0AA860F
:1052700014E0802912DAB28210E040290EDA0D2003
:1052800080012018828609E0402907DA0B2080017E
:10529000F7E7402902DAE8E78029E8DB0020F0BDE3
:1052A000C4130020F0B58DB0002501F019F9FCF70A
:1052B000CFFB059010213A4801F07CF90790FCF7EC
:1052C000C7FB04901021364801F01EF90690FCF748
:1052D000BFFB03901021324801F034F90190FCF734
:1052E000B7FB064610212E4801F044F90090FCF768
:1052F000AFFB2C4A04469068012108439060881E49
:10530000106129481061264B0021585C1070491C1F
:105310001029FADB1768FCF79BFB0B9001990098AA
:1053200002970190214F0091781921A1069B079ABD
:1053300000F066FE45190B98A11B001B019102901D
:10534000039A04990398B21A431A009208460599E1
:10535000421A781920A100F053FE441908A8FEF75C
:10536000F3F9264842680320C00302403819134667
:1053700023A100F045FE0419381926A1089A00F06F
:105380003FFE01193846FFF725FC01210D20FEF7ED
:1053900003FB24490320886000200DB0F0BD00000D
:1053A0001C6D00080030024001A00000E40700204E
:1053B0000D0A435243202025303458202025303414
:1053C00058202025303458202025303458202025DE
:1053D0003034580D0A00000074696D6520253034A2
:1053E000642020253034642020253034642020259A
:1053F0003034642020253034640D0A00001002404F
:105400004D61696E536F7572636520257820256440
:10541000200D0A00737973636C6B202564200D0ADC
:1054200000000000C000002030B50021174D0846E4
:10543000696042005219401C1181FF28F9DD0020EB
:105440000522134CD20143001B199B18401C998262
:105450001028F8DB00200922D20143001B199B18F9
:10546000401C9986FF28F8DD00201022C100091990
:1054700040310B8B401C93430B834028F6DB01200B
:10548000044928604882002030BD00003C11002003
:10549000C4130020781B002010B500210C480922FD
:1054A00001600C4B084692014400E418A418401C0B
:1054B000A1861028F8DB0020012292024400E418A3
:1054C000A418401CA1820828F8DB002010BD0000B1
:1054D0003C110020C413002010B5402802DB00203E
:1054E000C04310BD0B4BC100CA18114640310C7EA1
:1054F000A4060DD54000C0180B2300249B01C01842
:105500008486054800685065088B202290430883F4
:10551000002010BDC4130020E007002010B5FCF7E8
:105520006BFBFCF71DFF10BD70B594B030216846D1
:10553000FBF756FE0024022501260E94E80309908D
:10554000009605200F94C0040D9401960A900C94C7
:1055500008950B956846FCF7F1FC002803D08621DE
:1055600015A000F04BFD07200C900E9401210D9525
:105570000F940CA8FCF706FC002803D092210EA083
:1055800000F03CFD109610A81296FCF785FB002851
:1055900003D0A12108A000F031FD4B208001FCF7D1
:1055A000C7FE0420FCF77EFE00221146501EFCF7C9
:1055B0006FFB14B070BD00002E2E5C5372635C4212
:1055C00053502E630000000013480168012211436C
:1055D00001604168114A114041600168104A114060
:1055E00001600168012292049143016041683F22F9
:1055F000120491434160C16A09090901C162016B4A
:10560000FF22143291430163416B49084900416311
:105610000021816070470000001002400CB8FF08B4
:10562000FFFFF6FE04480169C907C90F02D0012136
:10563000C9430161704700000010004070B51B4C69
:10564000E0691B498006C00F11D01A4A0120106082
:10565000194A10600869401C0861A28C4868401C07
:105660004860174B154D18682A54401C1860E069B3
:105670000007C00F04D008202062C869401CC86120
:105680002068C006C00F07D0E069C006C00F03D075
:105690001020206200F01EF9E0694006C00F03D020
:1056A0004020206200F056F970BD00000038014033
:1056B000E4080020E8000020EC0000200C0A002094
:1056C000E000002010B5104CE069E0690007C00F51
:1056D00005D0082020620D48C169491CC1612068BD
:1056E000C006C00F07D0E069C006C00F03D010206D
:1056F000206200F07FF9E0694006C00F03D040202F
:10570000206200F0C7F910BD004400407809002075
:10571000F8B55E4CE0698006C00F09D0A08C5C4AE9
:10572000C1B21068FF2803D25A4B1954401C1060B4
:10573000E06900250006C00F8026002810D05649D9
:10574000564A08681368984205D30D6015602068B2
:10575000B043206004E0524A125C401C086022857D
:10576000E0690007C00F01D0082020622068C00651
:10577000C00F07D0E069C006C00F03D01020206220
:1057800000F090F9E06940274006C00F002802D0E1
:10579000276200F093F9434CE0698006C00F09D0FE
:1057A000A08C414AC1B21068FF2803D23F4B195464
:1057B000401C1060E0690006C00F10D03C493D4B12
:1057C00008681A68904205D30D601D602068B043D8
:1057D000206004E0384A125C401C08602285E069C1
:1057E0000007C00F01D0082020622068C006C00F4B
:1057F00007D0E069C006C00F03D01020206200F07F
:1058000075F9E0694006C00F02D0276200F07AF90E
:105810002A4CE0698006C00F09D0A08C284AC1B28A
:1058200010683F2803D2274B1954401C1060E069D0
:105830000006C00F10D02449244B08681A68904213
:1058400005D30D601D602068B043206004E0204A4D
:10585000125C401C08602285E0690007C00F01D07F
:10586000082020622068C006C00F07D0E069C0068B
:10587000C00F03D01020206200F05CF9E069400600
:10588000C00F02D0276200F061F9F8BD0048004067
:1058900074010020141E0020A001002078010020C7
:1058A000541D0020005000407C010020141F0020E7
:1058B000A401002080010020941D0020001401405C
:1058C0008401002014200020A8010020880100206D
:1058D000D41D00200548416A491C416204490968F9
:1058E000002901DD0121C16770470000E4080020A4
:1058F000E0000020F8B5144D0C460646022128466B
:10590000FDF73AFE10200090104B32460221284647
:10591000FDF71CFE224602212846FDF75FFE02210C
:105920002846FDF735FE0A48046301214172022131
:105930002846FDF739FE0548283881688022114342
:1059400081602046F8BD0000000002402838014078
:10595000E40800200248016A491C01627047000007
:10596000E408002010B50A48407A00280DD1084C00
:10597000206F5834002808D12046FBF7BFFF0146AE
:10598000E26820688018FFF7B5FF002010BD000016
:10599000E4080020F8B5144D0C46064605212846BB
:1059A000FDF7EAFD002000903346104A0521284605
:1059B000FDF7CCFD224605212846FDF70FFE052107
:1059C0002846FDF7E5FD0A4844630121817205215F
:1059D0002846FDF7E9FD0548243881684022114337
:1059E00081600020F8BD0000000002402444004017
:1059F000780900200A480B4900794058802180B27C
:105A0000081A0949012208600849CA674A6A521CF3
:105A10004A62002803DD01200549000748607047FD
:105A2000F46D000804000240E40000207809002022
:105A300000ED00E0F8B5144D0C460646042128465A
:105A4000FDF79AFD10200090104B324604212846A5
:105A5000FDF77CFD224604212846FDF7BFFD042109
:105A60002846FDF795FD0A4804630121417204218F
:105A70002846FDF799FD05482838816880221143A2
:105A800081602046F8BD000000000240284400402C
:105A9000780900200248016A491C01627047000031
:105AA0007809002003484068002802D002490120FC
:105AB000C867704770010020981B002070470000E5
:105AC00010B50C460A4601460548FBF770FB054831
:105AD00084600548016880221143016010BD000008
:105AE000541D002070010020004800400348C06899
:105AF000002802D002490120C867704770010020C9
:105B00002C1C00207047000010B50C460A460146C8
:105B10000548FBF74CFB05480461054801688022F5
:105B20001143016010BD0000941D00207001002091
:105B30000050004003484069002802D0024901207B
:105B4000C867704770010020C01C0020704700002B
:105B500010B50C460A4601460548FBF728FB0548E8
:105B600084610548016880221143016010BD000076
:105B7000D41D0020700100200014014010B5054C18
:105B80000A46638821465B1C4380FBF7A7FD002083
:105B900010BD0000007C000870B50C460B49411890
:105BA000002B08D00A4D4519012B03D0094B9B8AC5
:105BB000002B00D129468005204603D000F042F892
:105BC000002070BDFBF78AFDFAE7000000800008A6
:105BD00000A00008781B0020F8B54188174A491C2E
:105BE0004180154901807E2100250A52ED43802322
:105BF00000221146124C002659430C19314603E08D
:105C0000675CFF2F04D1491C9942F9DB002E03D0B9
:105C1000521C082AEDDB00E01546082D06D2084983
:105C20005D436918802200F00DF803E080220449EA
:105C3000FBF754FD0020F8BDAA550000A55A00004E
:105C400000C00008F7B50D460646FBF7BDFF0298F9
:105C50000024870807E0A0003258411900230220E1
:105C6000FBF774FF641CA742F5D802987C00470834
:105C700007E06000325A411900230120FBF766FF5C
:105C8000641CA742F5D8FBF757FFFEBDF7B588B0F7
:105C90000020069009980188C34881420FD10998D5
:105CA0008078C0070BD10998C178022907D3808872
:105CB000420809980092C0884008824202DB002016
:105CC0000BB0F0BD0291801A491EFBF725FA059032
:105CD0000898002870D1B5488168491C002481606B
:105CE00092E0600021180998009A0818059961430C
:105CF0008D18AE490A69521C0A61872189018D42BB
:105D000002DAAA4A01211170A9496A18A9498A42EE
:105D100024D2017BC07A890180080E182D20C00191
:105D2000281A074600F0B2FF70430190384600F091
:105D3000E3FB9E4F70433A6A84460C20134643436C
:105D40009D4819188E60019EC65060464860C72A5B
:105D500001DA521C3A62B969491CB961E12080013B
:105D6000854250DD91480078012848D18F4B1A6A4E
:105D7000002A44DD914D68422E46002117E00C2395
:105D80000F465F438C4BFB189C469B688C4FBB4275
:105D90000CDB63465B68002B03DDAB4206DA1D4675
:105DA00004E0002B02DA834200DD1846491C9142D0
:105DB000E5DB00218C4609E02CE00C230F465F4315
:105DC0007D4BDB59B34200DA1E46491C9142F4DB9D
:105DD000002D09D0002807D07D2128180901FBF7E4
:105DE0009BF9FBF712FA84466046FBF719FA6F4DF0
:105DF0007D21A862C9003046FBF78EF968636B48C5
:105E0000002101700162641C0298844202DA282C8D
:105E100000DA66E7089801287ED16448C168491C09
:105E20000024C160ADE0600021180998009A0818AC
:105E3000059961438D185D494A69521C4A61872161
:105E400089018D4202DA594A0121517058496A1874
:105E500058498A4223D2017BC07A890180080E18F2
:105E60002D20C001281A019000F010FF074677434B
:105E7000019800F041FB02464C480C21406A514B0E
:105E800084464843C1188E601F5072434A60604682
:105E90004649401C48620846C069401CC861E12070
:105EA000800185426CDD41484078012864D13F4A39
:105EB000506A049000285FDD002003903F48424B69
:105EC00041420191844600213E4F1CE00C220D46C8
:105ED0005543EE19B2681E2A14DB9A4201DA1346C2
:105EE00003917A59824200DA10467268002A03DD73
:105EF000624507DA944605E0002A03DA019DAA42CA
:105F000000DD0192491C049A9142DFDB00231D460B
:105F10001A4619462D4E00E039E08619079616E01C
:105F20000C270E467E43274FF719BF681E2F0DDB47
:105F3000244FBF59079EB74205DD052B06DD052A14
:105F400004DA6D1C02E0002D2BD0521C491C049E6B
:105F5000B142E5DB7D27FF00144E3946FBF7DCF844
:105F6000706303980C21484316494018406839462D
:105F7000FBF7D2F8B563F0620C4900204870486224
:105F8000641C0298844202DA282C00DA4BE70749A5
:105F90008A6B486B8018C20F10184010086306986F
:105FA0008EE65B1CD2E70000AA550000000200202C
:105FB0003FDEFFFF7F1600005822002040420F0006
:105FC00088130000B82B0020FFE0F50550C3000047
:105FD00010B5040001D0601C03D102210648FFF770
:105FE0006FFD012C01D0641C03D102210248FFF790
:105FF0008BFD002010BD000002020020FEE7000023
:106000000FB410B504A9074B02AA039800F028F8B2
:10601000044602A9002000F05DFA204610BC08BC2E
:1060200004B01847D564000830B47446641E25785F
:10603000641CAB4200D21D46635D5B00E31830BCBC
:10604000184702E008C8121F08C1002AFAD1704799
:106050007047002001E001C1121F002AFBD17047E8
:10606000FFB591B00F460546002606E025280AD068
:10607000149A139990476D1C761C28780028F5D146
:10608000304615B0F0BD002400940121F34A02947B
:1060900000E004436D1C2B780846203B98401042DA
:1060A000F7D128782A280ED0022128780246303AE3
:1060B000092A15D8009A0A235A43303A80180C430B
:1060C0006D1C0090F1E701CF0090002805DA012057
:1060D00040030443009840420090022004436D1C9A
:1060E00028782E2815D10420044368786D1C2A28AE
:1060F0000AD101CF6D1C02900BE002990A22514394
:10610000303940186D1C0290287801463039092931
:10611000F3D928786C2810D006DC4C281AD06828CF
:106120000ED06A2817D104E0742813D07A2812D12F
:1061300010E00120400504430CE00121090501E0C5
:10614000032109050C436978814203D10120000530
:1061500024186D1C6D1C287803906E281ED00CDC52
:10616000632831D004DC00288AD0582811D1B2E04D
:1061700064287BD069280CD178E073282DD004DC0A
:106180006F2870D0702804D1A7E075286CD07828CB
:106190006BD0149A13999047761C62E06002400F0E
:1061A000022807D003280AD0042838680AD00660DD
:1061B0003F1D56E03868F11706604160F8E738681F
:1061C0000680F5E70670F3E7387869460874002022
:1061D000487404A80390012003E03868039000206D
:1061E000C0433F1D61070FD5002101E00199491C03
:1061F000029A0191914213DA8142F7DB019A0399E5
:10620000895C0029F2D10BE0002101E00199491CD1
:1062100001918142FADB019A0399895C0029F5D149
:1062200001990098139A401A00902146149B00F09F
:106230003BF901998019461807E003980399007803
:10624000491C0391149A139990470198401E01909C
:10625000401CF2D12146149B139A009800F014F9C7
:1062600086196D1C09E741E033E034E00A20002183
:10627000049005916002410F022905D001CFC21799
:106280009446032905D007E0FF1DFF08FF0003CF58
:1062900006E000B2C2179446042902D140B2C117E9
:1062A0008C4600226146944506DA0A4600214042A7
:1062B00091418C462D2102E0210504D52B216A460F
:1062C0001176012103E0E10701D02021F7E70191D8
:1062D00054E00A200BE0102009E010200490002177
:1062E0000420044308200591029003E008200021C7
:1062F000059104906002410F022905D001CF0022D0
:106300009446032906D006E0FF1DFF08FF0003CFD7
:106310008C4603E080B2042900D1C0B20021019173
:1063200021072BD50399702906D0049A1021059BCB
:106330004A401A4305D00EE040216A4611760121F9
:1063400008E06146014306D030216A461176039980
:10635000517602210191049A0821059B4A401A4373
:106360000CD16146014301D1610707D530216A464E
:106370001176012101910299491E02910399582930
:1063800004D037A103910FA90F910DE039A1F9E7CE
:106390006146059B049AFAF75CFF039B8C469B5C65
:1063A0000F9A521E0F92137061460143F0D10F985D
:1063B00007A9081A20300390600704D501200004C3
:1063C0008443029801E0012002900399884201DD94
:1063D000401A00E000204118029001980918009826
:1063E000401A0090E00306D42146149B139A0098AB
:1063F00000F05AF886190020049008E006A9085C0D
:10640000149A139990470498401C761C04900199A3
:106410008842F3DBE0030CD52146149B139A0098C5
:1064200000F042F8861904E0149A3020139990473E
:10643000761C0299481E02900029F5DC08E00F98AE
:106440000F990078491C0F91149A13999047761C64
:106450000399481E03900029F1DCFBE6092801009E
:1064600030313233343536373839616263646566CA
:10647000000000003031323334353637383941428C
:106480004344454600000000F8B5044600251E467A
:106490001746880404D405E039462020B0476D1C17
:1064A000641EF9D52846F8BDFFB50446002581B025
:1064B0001E46C80301D5302700E02027880404D5F4
:1064C00005E038460399B0476D1C641EF9D528468F
:1064D00005B0F0BD0A68531C0B60107070470000D7
:1064E00010B50A2101A0FEF775FB10BD1B5B324AF7
:1064F0001B5B303B304800002D2110B5C90140180E
:1065000000F0C4FB10BD000030B503460B48002965
:1065100000D101210A4C491E0ED31A7850400022A6
:10652000C50702D04008604000E04008521CD2B2CB
:10653000082AF5D35B1CEEE730BD0000FFFF00002A
:1065400001A0000070B50A4DFF23EE1D1A46F93672
:1065500005E0047854402A5D5A40335D401C0C46E7
:10656000491E89B2002CF4D11802104370BD0000FE
:10657000FA6F000870B504460C4800220C4E11E07A
:106580002378521C1D4645402D07ED0E755B000912
:106590004540180968400007C00E305A2B09584082
:1065A00092B2641C8A42EBD370BD0000FFFF000072
:1065B0002C6D000810B5084A084B07E004785440D9
:1065C0002406E40D1C5B120A6240401C491EF5D2F1
:1065D000D04380B210BD0000FFFF0000FA6D00083C
:1065E00006C00021016041608160C160012202613A
:1065F00041610846704700008AB0002080F310888F
:10660000FE4F0126FF203E830530FD4B8022009087
:10661000991AFC48FBF7F0FE4020FB4B0246191A82
:106620000090FA48FBF7E8FEFBF7EEFA0021F84A83
:106630000D466020484380184560856005614561CE
:106640008561C561056285624562C562491C056355
:106650000929EEDBEF4CF0482567C06A6066EF4819
:106660000068A066EE48406AE066FEF75DFFEE490E
:10667000EC480860FBF7D0FEFDF706FA0320039014
:10668000049501A902960595E848FDF70BF8FDF77A
:10669000E7F9FCF7D1FEE648FEF790FBD748068302
:1066A000FEF788FBA063E34960630E70E249E34AAA
:1066B0000E700107090FE24F11701F2805D0C006A8
:1066C00006D5E04806703D7005E0DF480670F8E743
:1066D000DC4805703E70DD480170DD49012008701E
:1066E000E121DC4849020160FDF766FAFDF7F6FAA0
:1066F000FDF7B4FBD848006820210843D64908605C
:106700000868102630430860FDF7F2FBD3480168A3
:10671000202211430160016831430160FDF732FC22
:10672000CF480168202211430160016831430160B4
:10673000FDF744F9FDF7FCF9FDF714FAC9480168C3
:10674000012211430160C848016820221143016001
:1067500001683143016001684022114301608021DA
:10676000C248FFF717F9C248016831430160016868
:106770004022114301600A20FBF780F90120FEF757
:1067800021FD0020FEF708FD0020FEF71FFA012082
:10679000FAF79AFF0020FEF70BFDFEF783FDFBF7EB
:1067A00057F96066954D002028826882A048C0880D
:1067B0002882288A01280AD1FBF7D8FD208F2021C2
:1067C00008406882688A002801D0FEF72DFEA94E95
:1067D0005A2070840020C043FFF7FAFB0121A6482D
:1067E0008902411808910F218901411809911B2143
:1067F000890145180F21C901401800909F4F0020C2
:10680000387001207870FBF723F93861FBF7EEF957
:106810000790FEF7CFFA07467848008AC0070BD0EA
:10682000B806208F04D5800606D4FEF7FDFD03E0F0
:10683000800601D5FEF730FEA7630798E0630920C4
:10684000C00600690099888478480069C8848C482B
:10685000006908858B4800694885FBF787F8307523
:10686000FBF7F6F8854F786187480068002801D06B
:106870000020B082206CC006C00E02281CD1FAF79E
:10688000ABFD8148016800290ED00021B1827F490B
:106890000A68002A10D1006808607D4800687D49B8
:1068A0000860FDF709FE07E078490A68002A03D06E
:1068B00000680860FDF718FE5048008A01280BD1D7
:1068C0004E48818A002927D07349B960C18A73482C
:1068D0000160B868FDF710FE606E79696166081A9C
:1068E000A066E16E884200D2E066216F884200D93E
:1068F0002067FBF7ADF8B86152480078002806D051
:1069000052480078002802D00220FBF7B3FE079817
:10691000800403D5012002E06149D6E700203870E9
:106920000798000501D5012000E000207870444858
:10693000007800281DD00220FCF7B2F8606C002817
:1069400001D158490870574801784078000208186A
:106950000899888254490868800401D5012000E024
:10696000002038700868000501D5012000E00020F3
:106970007870606C002801D0401E6064A06C002814
:1069800001D0401EA0641D48018B002934D07878C6
:10699000FEF718FC7878FEF7FFFB7878FEF7F0FB3F
:1069A0007878002801D1012000E00020FEF700FCEB
:1069B000FBF74EF8F8610998B18A81860898808AB9
:1069C000B086FBF745F83862FBF742F80A21786297
:1069D0000846FAF77BFB0020401C4028FCDB206CBB
:1069E0003249401C20640868002806DD054AD26F41
:1069F000002A02D082B25BE06CE08BE0781B0020C2
:106A0000D4200020E408002018220020780900206B
:106A10002C0C00204419002080F7FF1FD400002018
:106A20000010024010270000AC01002000040048C4
:106A300044130020D8010020D9010020F4000020D8
:106A4000F1000020F000002028010020FB000020C1
:106A5000F5000020D8000020004800400050004011
:106A60000014014000100040003801408C0A002052
:106A70000044004004160020C4130020B001002090
:106A800000080048000C0048640100206801002054
:106A90008C0100206C01002000A000083C010020B7
:106AA000008000080C0B00200C010020E0000020FA
:106AB00056490120FDF7CEFA002805D05448534925
:106AC00002680120FCF728F951490020086051496B
:106AD000C86732E0008A01280FD0606C002810D00F
:106AE0007878FEF76FFBA06C00280CD07878FEF762
:106AF00053FB7878FEF744FB57E7474800680028C7
:106B0000EFD03878EDE70020FEF746FB0020FEF7D7
:106B100037FB48E74149786888420DD940484168C9
:106B200001221205114341604168520003235B05B5
:106B300099431143416001E0401C78603948007876
:106B4000002802D00020FAF799FF374FF86F00288D
:106B500008D0364801783648FEF7F6F93349002068
:106B60000860F86733483449407D0870FEF7ACF997
:106B70003248007870753248C06F00280CD0A88861
:106B8000304F401CA880304900203A68FFF77EF85B
:106B900000202B493860C8672C480088E8802C48C2
:106BA000008828812B48008868812B48C06F002806
:106BB0000CD0A88A294F401CA882294901203A6894
:106BC000FFF764F8002024493860C867254800882A
:106BD000E882254800882883244800886883244860
:106BE0000088A88423480088E884234800882885F2
:106BF00022480088688522480088A885B08EFDF765
:106C0000E5FF21491F480860F8E500000C0A002054
:106C1000E0000020E40800203C110020C02709000B
:106C200000380140F1000020C01C00208401002039
:106C30001420002024160020DA010020DB010020AF
:106C4000981B002074010020141E00200802002060
:106C500010020020180200202C1C00207C010020C3
:106C6000141F00200C020020140200201C0200202F
:106C7000280200202C0200203002002034020020D4
:106C800038020020AAAA00000030004010B52D21D3
:106C90004902FAF741FAC817800E4018821180099C
:106CA0008001081A1B4B40245A2A04DA91005A58D2
:106CB000C918496808E0B42A0FDAB421891A890092
:106CC0005A58C9188039C96F231A534348431818B2
:106CD000C117890E0818801110BDFF210F318A429B
:106CE00006DA0D49920051185A58C918496807E048
:106CF000FF216931891A89005A58C9188039C96F2A
:106D0000231A534348431818C117890E08188011D5
:106D1000404210BD3C02002030FDFFFF11223344F1
:106D20005566778899AABBCCDDEEFF00000001CC48
:106D300001D8001401F0003C002801E401A0006C1F
:106D4000007801B40050019C018800440111070142
:106D5000000100010401000000000000000000002C
:106D600000000600AA55000000010000000000001D
:106D70000100010000090000000000000000020006
:106D800000000009000000000000000000000000FA
:106D900000000000000000000000000010101010B3
:106DA00010101010101010101010101010002000F3
:106DB00030004000500060000300000004000000AC
:106DC00005000000060000000700000008000000A9
:106DD000090000000A0000000B0000000C00000089
:106DE0001100A55AAA550000000000000000000094
:106DF00000000000081C30445800000089111223D4
:106E00009B322446AD573665BF74488CC19D5AAF3E
:106E1000D3BE6CCAE5DB7EE9F7F881100801933335
:106E20001A22A5562C47B7753E64C99C408DDBBF1E
:106E300052AEEDDA64CBFFF976E802218B30100216
:106E400099132667AF763444BD554AADC3BC588EFE
:106E5000D19F6EEBE7FA7CC8F5D983310A209112F5
:106E60001803A7772E66B5543C45CBBD42ACD99EDE
:106E7000508FEFFB66EAFDD874C904428D5316614A
:106E80009F702004A9153227BB364CCEC5DF5EEDBE
:106E9000D7FC6888E1997AABF3BA85520C439771B5
:106EA0001E60A1142805B3373A26CDDE44CFDFFD9E
:106EB00056ECE9986089FBBB72AA06638F72144096
:106EC0009D512225AB343006B9174EEFC7FE5CCC7E
:106ED000D5DD6AA9E3B8788AF19B87730E62955075
:106EE0001C41A3352A24B1163807CFFF46EEDDDC5E
:106EF00054CDEBB962A8F99A708B088481951AA7D2
:106F000093B62CC2A5D33EE1B7F04008C919522B65
:106F1000DB3A644EED5F766DFF7C899400859BB70C
:106F200012A6ADD224C3BFF136E0C1184809D33B45
:106F30005A2AE55E6C4FF77D7E6C0AA583B41886ED
:106F400091972EE3A7F23CC0B5D14229CB38500A25
:106F5000D91B666FEF7E744CFD5D8BB502A49996CC
:106F60001087AFF326E2BDD034C1C3394A28D11A05
:106F7000580BE77F6E6EF55C7C4D0CC685D71EE521
:106F800097F42880A1913AA3B3B2444ACD5B5669E5
:106F9000DF78600CE91D722FFB3E8DD604C79FF58C
:106FA00016E4A9902081BBB332A2C55A4C4BD779C5
:106FB0005E68E11C680DF33F7A2E0EE787F61CC46D
:106FC00095D52AA1A3B03882B193466BCF7A5448A5
:106FD000DD59622DEB3C700EF91F8FF706E69DD44C
:106FE00014C5ABB122A0B9923083C77B4E6AD55885
:106FF0005C49E33D6A2CF11E780F00C1814001C05D
:10700000804101C0804100C1814001C0804100C178
:10701000814000C1814001C0804101C0804100C168
:10702000814000C1814001C0804100C1814001C058
:10703000804101C0804100C1814001C0804100C148
:10704000814000C1814001C0804100C1814001C038
:10705000804101C0804100C1814000C1814001C028
:10706000804101C0804100C1814001C0804100C118
:10707000814000C1814001C0804101C0804100C108
:10708000814000C1814001C0804100C1814001C0F8
:10709000804101C0804100C1814000C1814001C0E8
:1070A000804101C0804100C1814001C0804100C1D8
:1070B000814000C1814001C0804100C1814001C0C8
:1070C000804101C0804100C1814001C0804100C1B8
:1070D000814000C1814001C0804101C0804100C1A8
:1070E000814000C1814001C0804100C1814001C098
:1070F000804101C0804100C1814000C0C101C30383
:1071000002C2C60607C705C5C404CC0C0DCD0FCFFF
:10711000CE0E0ACACB0BC90908C8D81819D91BDB6F
:10712000DA1A1EDEDF1FDD1D1CDC14D4D515D717BF
:1071300016D6D21213D311D1D010F03031F133F36F
:10714000F23236F6F737F53534F43CFCFD3DFF3FBF
:107150003EFEFA3A3BFB39F9F83828E8E929EB2BEF
:107160002AEAEE2E2FEF2DEDEC2CE42425E527E77F
:10717000E62622E2E323E12120E0A06061A163A3EF
:10718000A26266A6A767A56564A46CACAD6DAF6F7F
:107190006EAEAA6A6BAB69A9A86878B8B979BB7BEF
:1071A0007ABABE7E7FBF7DBDBC7CB47475B577B73F
:1071B000B67672B2B373B17170B05090915193536F
:1071C000529296565797559594549C5C5D9D5F9F3F
:1071D0009E5E5A9A9B5B99595898884849894B8B6F
:1071E0008A4A4E8E8F4F8D4D4C8C448485458747FF
:1071F00046868242438341818040081C30445808BF
:107200001C3044580000000000000000010203048C
:107210000607080900000000010203043C72000890
:10722000C00000202407000078130008A87500089B
:10723000E40700205431000052600008D2000162CF
:107240000109000810C2010040420F000131220074
:10725000052F0101010001D2014612976712FF01BB
:10726000026500019310270D0004448000085600B9
:107270000538A560A5653E12118B12238F12349339
:1072800012469712579B12699F167A20128B5E1630
:107290009C8B16AE8F16BF2C16D03016E13412F22E
:1072A000CC160341121404122404123504124604AD
:1072B00012560412660412770412870412970412FD
:1072C000A70412B60412C60412D50412E50412F47F
:1072D0003C1006030200001204122104122F0412B3
:1072E0003E04124C04125A041268041275041283EC
:1072F00004129004129D0412AA0412B70412C304CB
:1073000012CF0412DB0412E70412F30412FE4C1332
:107310000903901104121F04122904123304123DB0
:1073200004124704125004125904126204126B042E
:10733000127304127B04128304128A041292041240
:107340009904129F0412A60412AC0412B20412B7DC
:107350000412BC0412C10412C60412CA0412CE04E0
:1073600012D20412D60412D90412DC0412DE041262
:10737000E10412E30412E40412E60452E70492E882
:1073800004611452E62852E33852DE4852D958526A
:10739000D26852CA7852C18852B79852ACA8529F4C
:1073A000B85292C85283D85273E85262F8565008C5
:1073B000563D185629282530253856FE4856E75898
:1073C00056CF6856B778569D885683985668A85603
:1073D0004CB8562FC825D025D856F4E856D5F85ABB
:1073E000B6085A97185A77285A56385A35482950A5
:1073F00029585AF2685AD0785AAE885A8B985A69E6
:10740000A85A46B85A23C82D37041EEFD10312DDFF
:107410000412CC0412BA0412A904129704128604AE
:107420001275041264041252041241041230041240
:107430001F041E0E05041006FDFEFFFFEC0412DC07
:107440000412CB0412BA0412AA04129A0412890478
:10745000127904126904125904124A04123A0412ED
:107460002B04121B04120C3C1006FDFDFFFFEE0462
:1074700012DF0412D10412C20412B40412A60412C0
:107480009804128B04127D041270041263041256C5
:1074900004124904123D0412310412250412190485
:1074A000120D0412024C13F7FC90110412E10412A5
:1074B000D70412CD0412C30412B90412B00412A7E7
:1074C00004129E04129504128D04128504127D0488
:1074D000127604126E04126704126104125A041226
:1074E0005404124E04124904124404123F04123A86
:1074F00004123604123204122E04122A0412270433
:10750000122404122204121F04121D04121C04125D
:107510001A045219049218046114521A28521D3880
:10752000522248522758522E68523678523F88527B
:1075300049985254A85261B8526EC8527DD8528DA3
:10754000E8529EF856B00856C31856D7282530255D
:107550003856024856195856316856497856638845
:10756000567D985698A856B4B856D1C825D025D877
:10757000560CE8562BF85A4A085A69185A89285A5C
:10758000AA385ACB48295029585A0E685A30785A86
:1075900052885A75985A97A85ABAB829C029C83C2F
:0875A00004001BB79B0600006C
:04000005080010B926
:00000001FF
